:100000000C942A001895000018950000189500001F
:100010000C94170B18950000189500001895000017
:10002000189500000C94C205189500001895000062
:10003000189500001895000018950000189500000C
:1000400018950000189500001895000018950000FC
:10005000189500008FE58DBFC0E2E0E24E2E84E0EF
:100060008EBFD4E0F4E05F2EA89584B7082E877F7A
:1000700084BF88E1992781BD91BDEEEFF3E0A0E652
:10008000B0E088278D933197E9F70E94EC09662448
:1000900088E082BD85E085BD89B7806489BF85E041
:1000A00083BFAFE6B0E0E6EBF8E10E94AF0A0E9442
:1000B000690A789480E08093C20080E080932601F2
:1000C00080E080938A0181E08093C30080E0809388
:1000D000270180E080938B0181E08093C40081E060
:1000E0008093280180E080938C0182E08093C5009A
:1000F00081E08093290181E080938D0185E08093E8
:10010000C60080E080932A0185E080938E0185E01F
:100110008093C70082E080932B0185E080938F015C
:1001200087E08093C80080E080932C0187E0809373
:10013000900187E08093C90083E080932D0183E0E4
:100140008093910186E08093CA0087E080932E011E
:1001500087E08093920187E08093CB0087E08093D3
:100160002F0187E08093930180E08093CC0080E0B2
:100170008093300180E08093940180E08093CD00F3
:1001800081E08093310180E08093950182E080934B
:10019000CE0080E08093320181E08093960182E07E
:1001A0008093CF0082E08093330182E080939701B7
:1001B00082E08093D00085E08093340182E08093D8
:1001C000980182E08093D10087E08093350182E03E
:1001D0008093990185E08093D20085E08093360179
:1001E00085E080939A0185E08093D30085E0809339
:1001F000370187E080939B0187E08093D40086E0FD
:100200008093380187E080939C0187E08093D5003C
:1002100087E08093390187E080939D0180E080939F
:10022000D60080E080933A0180E080939E0180E0D8
:100230008093D70080E080933B0181E080939F0111
:1002400084E08093D80080E080933C0182E080933A
:10025000A00181E08093D90080E080933D0185E09A
:100260008093A10182E08093DA0083E080933E01D5
:1002700081E08093A20184E08093DB0084E080939E
:100280003F0187E08093A30186E08093DC0086E055
:100290008093400186E08093A40187E08093DD0095
:1002A00086E08093410186E08093A50187E08093FA
:1002B000DE0087E08093420186E08093A60187E01C
:1002C0008093DF0087E08093430187E08093A7015C
:1002D00080E08093E00080E08093440180E08093A0
:1002E000A80182E08093E10080E08093450180E0F6
:1002F0008093A90181E08093E20080E08093460131
:1003000081E08093AA0180E08093E30080E0809305
:10031000470187E08093AB0186E08093E40082E0B0
:100320008093480182E08093AC0187E08093E500F0
:1003300085E08093490180E08093AD0187E0809360
:10034000E60087E080934A0180E08093AE0187E079
:100350008093E70084E080934B0187E08093AF01B6
:1003600085E08093E80087E080934C0187E08093EC
:10037000B00187E08093E90087E080934D0187E03A
:100380008093B10180E08093EA0080E080934E0189
:1003900080E08093B20180E08093EB0082E0809364
:1003A0004F0180E08093B30182E08093EC0081E014
:1003B0008093500180E08093B40184E08093ED004D
:1003C00083E08093510180E08093B50185E08093C4
:1003D000EE0084E08093520184E08093B60187E0D0
:1003E0008093EF0084E08093530182E08093B70113
:1003F00087E08093F00082E08093540185E0809351
:10040000B80186E08093F10087E08093550183E096
:100410008093B90187E08093F20085E080935601D4
:1004200087E08093BA0187E08093F30087E08093B0
:10043000570187E08093BB0180E08093F40080E067
:100440008093580180E08093BC0180E08093F500A8
:1004500080E08093590182E08093BD0182E0809327
:10046000F60080E080935A0182E08093BE0181E033
:100470008093F70082E080935B0184E08093BF016A
:1004800086E08093F80083E080935C0180E08093B5
:10049000C00186E08093F90086E080935D0181E0F1
:1004A0008093C10181E08093FA0083E080935E0134
:1004B00087E08093C20183E08093FB0087E0809314
:1004C0005F0186E08093C30187E08093FC0087E0B2
:1004D0008093600185E08093C40187E08093FD00F4
:1004E00087E08093610187E08093C50180E080937D
:1004F000FE0080E08093620180E08093C60184E08A
:100500008093FF0080E08093630180E08093C701C7
:1005100080E08093000183E08093640180E0809319
:10052000C80184E08093010182E08093650181E04D
:100530008093C90180E08093020187E08093660187
:1005400081E08093CA0182E08093030185E080937B
:10055000670183E08093CB0186E08093040187E00C
:100560008093680181E08093CC0185E08093050150
:1005700087E08093690185E08093CD0183E08093DB
:10058000060187E080936A0187E08093CE0187E0CF
:100590008093070187E080936B0187E08093CF0110
:1005A00080E08093080180E080936C0180E080937C
:1005B000D00180E08093090184E080936D0180E0A8
:1005C0008093D10181E080930A0180E080936E01E5
:1005D00082E08093D20182E080930B0184E08093DB
:1005E0006F0182E08093D30183E080930C0180E06F
:1005F0008093700186E08093D40182E080930D01A6
:1006000083E08093710186E08093D50184E080933C
:100610000E0187E08093720185E08093D60187E028
:1006200080930F0182E08093730187E08093D7016C
:1006300087E08093100183E08093740187E08093CA
:10064000D80187E08093110187E08093750187E0EE
:100650008093D90180E08093120180E0809376013D
:1006600080E08093DA0180E08093130180E0809342
:10067000770184E08093DB0180E08093140185E0C2
:100680008093780180E08093DC0184E08093150101
:1006900081E08093790184E08093DD0181E08093A3
:1006A000160183E080937A0181E08093DE0181E08E
:1006B0008093170185E080937B0185E08093DF01C3
:1006C00085E08093180181E080937C0187E080932E
:1006D000E00183E08093190185E080937D0187E04C
:1006E0008093E10187E080931A0187E080937E0187
:1006F00083E08093E20187E080931B0187E0809391
:100700007F0187E08093E30180E080931C0180E01B
:100710008093800180E08093E40180E080931D015C
:1007200082E08093810180E08093E50181E0809305
:100730001E0182E08093820180E08093E60180E0E8
:1007400080931F0183E08093830182E08093E7011F
:1007500084E08093200185E08093840184E080938D
:10076000E80186E08093210180E08093850187E0A5
:100770008093E90185E08093220187E080938601E0
:1007800082E08093EA0186E08093230185E08093F4
:10079000870187E08093EB0187E08093240185E067
:1007A0008093880187E08093EC0187E080932501A6
:1007B00087E08093890187E08093ED0180E080935A
:1007C000EE0180E08093520281E08093EF0180E0AF
:1007D0008093530281E08093F00181E08093540282
:1007E00087E08093F10180E08093550286E080935A
:1007F000F20183E08093560287E08093F30185E065
:100800008093570287E08093F40187E08093580239
:1008100080E08093F80180E080935C0280E0809328
:10082000F90181E080935D0282E08093FA0181E02A
:1008300080935E0282E08093FB0185E080935F02FB
:1008400087E08093FC0181E08093600285E08093E3
:10085000FD0187E08093610287E08093FE0187E0DD
:100860008093620280E08093020280E080936602BF
:1008700082E08093030280E08093670284E08093AB
:10088000040282E08093680285E08093050282E0A2
:100890008093690284E08093060287E080936A0275
:1008A00087E08093070283E080936B0287E0809368
:1008B000080287E080936C0280E080930C0280E065
:1008C0008093700280E080930D0282E08093710239
:1008D00085E080930E0280E08093720281E0809335
:1008E0000F0283E08093730285E08093100285E01D
:1008F0008093740286E08093110287E080937502F2
:1009000087E08093120287E08093760280E08093F4
:10091000160280E080937A0284E08093170280E0E0
:1009200080937B0283E08093180280E080937C02B6
:1009300086E08093190281E080937D0287E08093B6
:100940001A0282E080937E0283E080931B0287E09C
:1009500080937F0287E080931C0287E0809380026F
:1009600080E08093200280E08093840280E0809386
:10097000210284E08093850284E08093220284E057
:100980008093860281E08093230285E08093870232
:1009900086E08093240286E08093880287E080933B
:1009A000250283E08093890287E08093260287E016
:1009B00080938A0280E08093B60281E08093B70240
:1009C00083E08093B80287E08093B90280E080934F
:1009D000C00282E08093C10285E08093C20287E07A
:1009E0008093C30280E08093CA0284E08093CB02AC
:1009F00086E08093CC0287E08093CD028FEF8ABBA4
:100A000080E087BB8FE084BB80E08BBB84E090E01C
:100A1000A2EAB0E08D939C9381E090E0A8E7B0E07B
:100A20008D939C9381E090E0A0EAB0E08D939C933D
:100A300085E090E0A4EAB0E08D939C9380E0809301
:100A4000BB0082E08093BD000E94ED06A8E7B0E005
:100A50000D911C91003051E0150710F00C944905E0
:100A600088E085BBA8E7B0E0EBE3F0E042E00E945D
:100A7000DF09A0EAB0E0AD90BC90AAE7B0E0AA0C14
:100A8000BB1CAA0DBB1D0C9148E0040F05BB0C94C8
:100A9000590580E085BB8FEF8BBBA0EAB0E0AD903D
:100AA000BC90AAE7B0E0AA0CBB1CAA0DBB1D8C91A0
:100AB00085BB91E0A8E7B0E00E94B50AA0EAB0E0EB
:100AC0000E94E509A8E7B0E00D911C91003052E0CA
:100AD000150711F00C94780581E090E0A8E7B0E0EC
:100AE0008D939C9381E090E0A0EAB0E08D939C937D
:100AF000B998AAE1B3E09C9197FF04C0B19910C0E6
:100B00009F779C93B19B0CC082E09F9399270E9492
:100B1000510A9F91B19B04C090689C930E949608D3
:100B2000BA98AAE1B3E09C9196FF04C0B29910C0B4
:100B30009F7B9C93B29B0CC082E09F9399270E945D
:100B4000510A9F91B29B04C090649C930E94BA0882
:100B5000B898AAE1B3E09C9195FF04C0B09910C089
:100B60009F7D9C93B09B0CC082E09F9399270E942D
:100B7000510A9F91B09B04C090629C930E945009BF
:100B80000C9426050F921F922F923F924F925F92E4
:100B90007F92AF92BF920F931F932F933F934F93E8
:100BA0005F936F937F938F939F93AF93BF93CF93F5
:100BB000DF93EF93FF938FB78F93ACEBB0E08C9103
:100BC0008F5F8C930091BC00093010F00C944A06A2
:100BD0000091BB00013011F00C94080680E090E019
:100BE000ACE7B0E08D939C9380E090E0AEE7B0E09E
:100BF0008D939C9380E090E0A0E8B0E08D939C936F
:100C000080E090E0A2E8B0E08D939C930C944806BD
:100C1000023011F00C942C0680E090E0A4E8B0E0E3
:100C20008D939C9380E090E0A6E8B0E08D939C9338
:100C300080E090E0A8E8B0E08D939C9380E090E0A5
:100C4000AAE8B0E08D939C9380E090E0ACE8B0E03F
:100C50008D939C930C944806033011F00C94480635
:100C600082E090E0ACE7B0E08D939C9380E090E070
:100C7000A8E8B0E08D939C9380E090E0AAE8B0E013
:100C80008D939C9380E090E0ACE8B0E08D939C93D2
:100C90000C94C806AEEBB0E0AD90BB24A5EBB2E07F
:100CA000AA0DBB1D8C91ACE7B0E08D9388278C9387
:100CB000AFEBB0E0AD90BB24A1ECB0E0AA0DBB1D42
:100CC0008C91AEE7B0E08D9388278C93AFEBB0E0CA
:100CD000AD90BB24A5E2B1E0AA0DBB1D8C91A0E8AC
:100CE000B0E08D9388278C93AFEBB0E0AD90BB2440
:100CF000A9E8B1E0AA0DBB1D8C91A2E8B0E08D93EC
:100D000088278C93A0ECB0E0AD90BB24ADEEB1E0B1
:100D1000AA0DBB1D8C91A4E8B0E08D9388278C931D
:100D2000A0ECB0E0AD90BB24A1E5B2E0AA0DBB1DE4
:100D30008C91A6E8B0E08D9388278C93A1ECB0E06D
:100D4000AD90BB24A1ECB0E0AA0DBB1D8C91A8E82E
:100D5000B0E08D9388278C93A1ECB0E0AD90BB24DC
:100D6000A5E2B1E0AA0DBB1D8C91AAE8B0E08D937D
:100D700088278C93A1ECB0E0AD90BB24A9E8B1E04A
:100D8000AA0DBB1D8C91ACE8B0E08D9388278C93A5
:100D90000091BC00003111F00C94D10680E08093EA
:100DA000BC008F918FBFFF91EF91DF91CF91BF91E9
:100DB000AF919F918F917F916F915F914F913F91F3
:100DC0002F911F910F91BF90AF907F905F904F90A8
:100DD0003F902F901F900F901895A2EAB0E00E94CC
:100DE000E509A4EAB0E04D915C91A2EAB0E00D9172
:100DF0001C910417150711F00C9495080091BB0085
:100E0000033010F00C94C0070E94600AEFE6F0E097
:100E1000AEEAB0E00E94410CEEEAF0E001E0A6EAA2
:100E2000B0E00E944D0C82E0EEEAF0E001E00A93AF
:100E3000A8EAB0E00E94460C84E0EEEAF0E001E0AF
:100E40000A93AAEAB0E00E94460C85E0EEEAF0E0E0
:100E500001E00A93ACEAB0E00E94460CA6EAB0E0DA
:100E60000E940F0CAEEBB0E00C93A8EAB0E00E9439
:100E70000F0CAFEBB0E00C93AAEAB0E00E940F0CAD
:100E8000A0ECB0E00C93ACEAB0E00E940F0CA1EC37
:100E9000B0E00C9383E090E08A939A930E94F30968
:100EA000002F112F4AE050E00E94A50AAAE7B0E007
:100EB0000D931C930091BE0040917A00040FAEEB9D
:100EC000B0E00C938AE090E08A939A930E94F30931
:100ED000002F112F4AE050E00E94A50AAAE7B0E0D7
:100EE0000D931C930091BF0040917A00040FAFEB6B
:100EF000B0E00C9386E090E08A939A930E94F30905
:100F0000002F112F4AE050E00E94A50AAAE7B0E0A6
:100F10000D931C930091C00040917A00040FA0EC47
:100F2000B0E00C938AE090E08A939A930E94F309D0
:100F3000002F112F4AE050E00E94A50AAAE7B0E076
:100F40000D931C930091C10040917A00040FA1EC15
:100F5000B0E00C93AEEBB0E08C918F5F8C93AFEB75
:100F6000B0E08C918F5F8C93A0ECB0E08C918F5FA0
:100F70008C93A1ECB0E08C918F5F8C930C94110852
:100F8000AEEAB0E0E4EAF0E00E94BE0BEEEAF0E088
:100F9000A8E0B4E00E94410CE8E0F4E0AEEAB0E082
:100FA0001127222702E033270E94C40AEEEAF0E06C
:100FB00001E0AAEAB0E00E944D0CAEEAB0E00E9467
:100FC000550CEA2FFB2F32970FEFACEAB0E00E94EE
:100FD0004D0C8CE08093BE0080E08093BF00AAEAB5
:100FE000B0E00E940F0CA0ECB0E00C93ACEAB0E0D3
:100FF0000E940F0CA1ECB0E00C93AEEBB0E08C9132
:101000008F5F8C93AFEBB0E08C918F5F8C93A0ECF3
:10101000B0E08C918F5F8C93A1ECB0E08C918F5FEE
:101020008C93AEEBB0E0AD90BB24A5EBB2E0AA0D83
:10103000BB1D8C91ACE7B0E08D9388278C93AFEB10
:10104000B0E0AD90BB24A1ECB0E0AA0DBB1D8C912B
:10105000AEE7B0E08D9388278C93AFEBB0E0AD9016
:10106000BB24A5E2B1E0AA0DBB1D8C91A0E8B0E0C5
:101070008D9388278C93AFEBB0E0AD90BB24A9E8AB
:10108000B1E0AA0DBB1D8C91A2E8B0E08D9388273A
:101090008C93A0ECB0E0AD90BB24ADEEB1E0AA0D16
:1010A000BB1D8C91A4E8B0E08D9388278C93A0ECB5
:1010B000B0E0AD90BB24A1E5B2E0AA0DBB1D8C91C0
:1010C000A6E8B0E08D9388278C93A1ECB0E0AD90BA
:1010D000BB24A1ECB0E0AA0DBB1D8C91A8E8B0E048
:1010E0008D9388278C93A1ECB0E0AD90BB24A5E252
:1010F000B1E0AA0DBB1D8C91AAE8B0E08D938827C2
:101100008C93A1ECB0E0AD90BB24A9E8B1E0AA0DAE
:10111000BB1D8C91ACE8B0E08D9388278C9380E068
:1011200090E0A2EAB0E08D939C93089589B7816026
:1011300089BFA4EAB0E00D911C9141E050E0041B8E
:10114000150BA2EAB0E00D931C93ABEBB0E08C91D1
:101150008F5F8C930091BB00033018F011F00C945A
:10116000B3080C94B90880E08093BB0089B78E7FE8
:1011700089BF08950091BB00013011F00C94C7089D
:10118000A2E6B0E08C918F5F8C930C94DB08023068
:1011900011F00C94D208A1E6B0E08C918F5F8C9393
:1011A0000C94DB08033011F00C94DB08ADEBB0E0DD
:1011B0008C918F5F8C9300916200073118F011F0D1
:1011C0000C94E4080C94E70880E08093620000919E
:1011D00061000B3318F011F00C94F0080C94F30834
:1011E00080E0809361000091BD00013011F00C940B
:1011F000FF0881E090E0A4EAB0E08D939C93009119
:10120000BD00023011F00C940B0985E090E0A4EAD7
:10121000B0E08D939C930091BD00033011F00C94CD
:1012200017098AE090E0A4EAB0E08D939C930091C6
:10123000BD00043011F00C9423098FE090E0A4EA83
:10124000B0E08D939C930091BD00053011F00C949B
:101250002F098EE190E0A4EAB0E08D939C93009179
:10126000BD00063011F00C943B098CE390E0A4EA39
:10127000B0E08D939C930091BD00063018F011F002
:101280000C9444090C944D0981E08093BD0081E0E9
:1012900090E0A4EAB0E08D939C930E94FE0608952E
:1012A0000091BB00013011F00C945D098091620047
:1012B0008150809362000C947109023011F00C94FB
:1012C0006809809161008150809361000C947109DC
:1012D000033011F00C9471098091BD00815080930E
:1012E000BD00009162000F3F11F00C947A0987E174
:1012F00080936200009161000F3F11F00C9483090C
:101300008BE3809361000091BD00013011F00C94DB
:101310008F0981E090E0A4EAB0E08D939C93009166
:10132000BD00023011F00C949B0985E090E0A4EA26
:10133000B0E08D939C930091BD00033011F00C94AC
:10134000A7098AE090E0A4EAB0E08D939C93009115
:10135000BD00043011F00C94B3098FE090E0A4EAD2
:10136000B0E08D939C930091BD00053011F00C947A
:10137000BF098EE190E0A4EAB0E08D939C930091C8
:10138000BD00063011F00C94CB098CE390E0A4EA88
:10139000B0E08D939C930091BD000F3F11F00C9431
:1013A000DA0986E08093BD008CE390E0A4EAB0E027
:1013B0008D939C930E94FE060895EA2FFB2F8D913A
:1013C000809581934A95D9F70895ED91FC91EF5F4F
:1013D000FF4FFC93EE93089515E000E000931B038C
:1013E00010931C03089540911B0350911C030DEFB3
:1013F00013E40E94080A0D53114640E050E82ED035
:1014000000931B0310931C035991499127D0089511
:1014100009D00E94A50A00FC10D0089503D01ED068
:1014200001F8F9CF0024E89457FF02C009D068946E
:1014300000F80BD010F80124089502D009D00895C7
:10144000509540954F5F5F4F0895E89417FF0895BA
:10145000009510950F5F1F4F68940895352F242F26
:10146000E894452B11F468940895512F402F0027DC
:10147000112780E1440F551F001F111F021B130B82
:10148000416018F4020F131F4E7F8A9599F7089553
:101490003197F1F70895689462F80895E89462F836
:1014A0000895EF93FF93EE27E82BE92B31F0E0ED61
:1014B000F7E03197F1F70197D1F7FF91EF91089598
:1014C000A6E6B0E0E3E6F0E00E94950A33970C94BC
:1014D000830AEFE6F0E0A0E6B0E00E94710AADE01A
:1014E000BB27868197810E940D0B0D938381948188
:1014F0000E940D0B0D93808191810E940D0B0D9325
:101500000895EDE0FF2782810E94020B8AE38D930C
:1015100081810E94020B8AE38D9380810E94020BDD
:1015200088278C930895EDE0FF2781810E94020BAC
:101530008CE58D9380810E94020B8CE58D938281D6
:101540000E94020B88278D9308950F92B801469F41
:101550008001479F100D569F100D0F9008950E9417
:10156000C00A0D920020D9F70895903041F00D91F6
:101570001C91000F111F9A95E1F71C930E9308958B
:10158000C8953196002008952E2E3F2E99278191DF
:101590008D3209F093958823D1F79A95E22DF32D9A
:1015A000112361F0091718F011F0101B01C0191B6D
:1015B00028F021F080E28D931A95E9F780818D3231
:1015C00019F48D93319604C0222311F08BE28D9390
:1015D000091738F031F0091B21F080E38D930A954B
:1015E000E9F781918D938823E1F7332351F0EA2FB6
:1015F000FB2F319633958E9182933A95E1F78EE2E7
:101600008C93089500278A3018F08A500395FBCFF9
:10161000005D0D93805D8D93089580539053002756
:10162000813018F0065F8A95FBCF090F0895AF93BC
:10163000BF930F939F938F938FB78F93A0E6B0E0E4
:101640008C9183958D938C3309F03DC088278E93C0
:1016500011968C9183958D938C3309F034C0882733
:101660008E9311968C9183958D93883161F588279F
:101670008E9311968C9183958D939C910EE194306D
:1016800089F0963079F0993069F09B3059F00CE18F
:10169000923039F411969C911197937019F4039537
:1016A00001C00FE1801778F071F081E08E93119600
:1016B0008C9183958D938D3031F481E08E931196CA
:1016C0008C9183958C938F918FBF8F919F910F9168
:1016D000BF91AF910F921F922F923F924F925F92C4
:1016E0007F92AF92BF920F931F932F933F934F938D
:1016F0005F936F937F938F939F93AF93BF93CF939A
:10170000DF93EF93FF938FB78F930E94ED068F9136
:101710008FBFFF91EF91DF91CF91BF91AF919F91DB
:101720008F917F916F915F914F913F912F911F9179
:101730000F91BF90AF907F905F904F903F902F9010
:101740001F900F901895040F151F261F371F08951F
:10175000000F111F221F331F08950095109520952B
:1017600030950F5F1F4F2F4F3F4F0895019110810C
:101770000EC001911191219130810BC00191108116
:1017800017FF05C03FEF2FEF04C00081112722276C
:10179000332737FF03C0E1DF8DE28D93CF93DF93D3
:1017A000CF92DF92EF92AA24BB24CC24DD24EE2436
:1017B00040E2CAE0DD2755E093E38881890F87FD89
:1017C0009F7083FD907F891B89935A95A9F7C0DF8D
:1017D000AA1CBB1CCC1CDD1CEE1C4A9551F7E894DE
:1017E000EFE0FF2782910ED0EB30E0F71EF0689417
:1017F0008A2D0CD088278D93EF90DF90CF90DF91CA
:10180000CF910895982F829501D0892F8F70805D98
:1018100026F0803309F4089568948D930895002785
:101820001127222733271DD08A3328F4803318F05C
:1018300005D015D0F9CF0EF490CF089580538F9333
:10184000402F512F622F732F83DF82DF7CDF80DFF9
:101850008F919927080F191F291F391F08958D91FE
:101860000895E894FCDF8032E9F38B32D9F38930B4
:10187000C9F38D3211F46894F2CF089588278D93BF
:10188000089581918D938823E1F7089509919191AD
:10189000992351F08A95D9F7319781918D930A95C3
:1018A00019F08823D1F70895E9CF8FEF83959D91A3
:1018B0009923E1F7089531323A33343A3030000059
:00000001FF
